:020000040000FA
:04000000D2303A2898
:08000800A000030EA100831209
:100010008B1C32288B1031181428B11C3228643004
:10002000010203183128182800001628172818285C
:1000300019281A281B281C281D281E281F283110A3
:10004000B114A810031005190314AA0DA90DA80DC9
:10005000B00B322831152A08AF002908AE00280855
:10006000AD00B11081010B11210E8300A00E200EF6
:02007000090085
:0C007400203084008001840A80300402E7
:10008000031C3C281230B0007721850187018316BC
:100090000C30850587018312831605148715071612
:1000A0008312850187010730990000309A001030D3
:1000B00083168E008312603083168F008312003007
:1000C000831691009F008312C8308316810083122B
:1000D00031309000003083168C00831210308B007A
:1000E000831600309B001C141A088312BC00851D67
:1000F0000027831610309B001C141A088312BD00C1
:10010000CB2181018E018F010B118B100B108C0103
:100110008B1798203119AE20B30B96280310851940
:100120000314B90DF030390203190421C0238928C2
:100130006400311808000B1D08000B11B1103114B8
:100140001230B000051DA928321483160113831242
:100150000800321083160117831208003111013094
:10016000B7008B132030370783169B001C141A0826
:100170008312A400A500C030A506103037078316EF
:100180009B001C141A088312A30000303707831643
:100190009B001C141A088312A2008B17321CD6284D
:1001A00022090339A200A309A409A50922082D02E6
:1001B000031DFE2823082E02031DFE2824082F02FB
:1001C000031DFE2801303702031DE9283D143E14AB
:1001D000AB2102303702031DF028BD143E14AF21BD
:1001E00003303702031DF7283D153E14B3210430B8
:1001F0003702031DFE28BD153E14B721B70A05308E
:10020000370203180800B1283C1C08000130B60072
:10021000B300B400B500B70085018701B113982081
:10022000B30B2829031085190314B90DF0303902D6
:1002300003194F29B41F0710B40B28293708B60833
:100240000319B600031926290714B6039630B40023
:10025000311D0F293111321C32292D090339AD000E
:10026000AE09AF092F1CB1132F1C0F29B11B0F2989
:100270002E180F29B1178B1320303707BB002F081A
:10028000BA00622110303707BB002E08BA00622185
:1002900000303707BB002D08BA0062218B1785019B
:1002A0008701B70AB60105303702031C0F29CB219D
:1002B00008003E1C08003E101030BB003D08BA008C
:1002C000622108008B133A0883161C159A008312CA
:1002D0003B0883169B0055309D00AA309D009C145E
:1002E00064009C1870291C1183128B1708000030C1
:1002F0009500603084008B13831604089B001C1447
:100300001A0883128B178000840A68300402031CC9
:100310007B296430D5003424DC003C30EC00ED0057
:10032000EE00EF00EA146E30D50034240F39031DBF
:10033000080039240F39031D08003E240F39031D1E
:10034000080043240F39031D080083168711071284
:100350008312EA1008000130E800DA2108000230B8
:10036000E800DA2108000430E800DA21080008304B
:10037000E800DA2108001030E800DA210800203017
:10038000E800DA2108004030E800DA210800803077
:10039000E800DA210800EA178B13831670309B00FF
:1003A0001C141A0883128B17E800DA210430EB00C2
:1003B000EA130800E80803190800681CE7296730F9
:1003C000D5003424D1006830D5003424D200E81C94
:1003D000F1296730D5003924D1006830D50039249F
:1003E000D200681DFB296730D5003E24D10068305B
:1003F000D5003E24D200E81D052A6730D5004324ED
:10040000D1006830D5004324D200681E0F2A6A301C
:10041000D5003424D1006B30D5003424D200E81E3E
:10042000192A6A30D5003924D1006B30D50039241F
:10043000D200681F232A6A30D5003E24D1006B30D9
:10044000D5003E24D200E81F2D2A6A30D50043246F
:10045000D1006B30D5004324D200EA16D11A3D2AD0
:10046000511B3D2A511C3D2ADC1FEA125C1F3D2A0C
:10047000501C3D2AC01B3D2A0800EA1E4D2AEA1BDB
:100480004D2A511870308B1383169B001C141A08C8
:1004900083128B17680203190800D11A582A511BBE
:1004A000582A6A10511C582A5014051E6A14051641
:1004B000511C602A511A5016D11AC017511B5012E4
:1004C000EA1F672AD11A0800511B08006B2AD11AAB
:1004D000982A511B982A6530D500521A3424D21A12
:1004E0003924521B3E24D21B43245118C4006630C9
:1004F000D500521A3424D21A3924521B3E24D21B5E
:1005000043245118CC0052085118D70004306A18FF
:100510003230EA1B32305118C80051185C14EA1FFF
:10052000962A511C952A4403C00008005118C001A6
:1005300051187030BB006808E900BA006221BD01A3
:100540000800FD010730FF007B08FE0C0318AC2AF1
:10055000FF0BA52AFB0100340310B12AFE0C03187F
:10056000FB07FB0CFD0CFF0BAE2AFB0CFD0C003453
:1005700094019301093095008B138E018F018B1725
:10058000D6135608FB007508F51BFF3CFE00FE1352
:10059000A122FD0D7B0DF51FD607F51BD6025608CF
:0E05A000760793000318141408309500080025
:1007800002300F02031C0800EA1CDD2BA127F10830
:100790000319DD2B6E30D50071183424F11839247B
:1007A00071193E24F1194324E8006818AB21E818B8
:1007B000AF216819B321E819B7210730EB050330E1
:1007C0008A006B088207E82B1F2C202C212C222C5E
:1007D000501C2D2C4008D500571A3424D71A392420
:1007E000571B3E24D71B4324D6006108F500600840
:1007F000F6005C1CB822C80B2D2C4C085C18053088
:10080000C8005C1CC00A5C1044084002031C2D2C6C
:10081000C01B0E2C501E0E2CC0012D2C7A18152C2E
:100820007A140930C800C0032D2C5012DC180512B0
:100830005C1950105C1DC0035C1DC0172D2C2D2CA5
:100840002D2C2D2C071C262C07102D2CE908031904
:100850002D2C07140310E90C2D2CEB0A05306B022C
:100860000318EB018F01080005308A00D5135508E5
:10087000820005308A00D5175508820006308A00AC
:10088000D5135508820006308A00D5175508820016
:100A00000034013403340434053406340834093422
:100A10000A340B340D340E340F34113412341334C1
:100A2000143416341734183419341B341C341D3460
:100A30001E342034213422342434253426342734FF
:100A400029342A342B342C342E342F34303432349D
:100A50003334343435343734383439343A343C343C
:100A60003D343E34403441344234433445344634DA
:100A7000473448344A344B344C344D344F3450347A
:100A800051345334543455345634583459345A3418
:100A90005B345D345E345F346134623463346434B7
:100AA00066346734683469346B346C346D346E3456
:100AB00070347134723474347534763478347A34F2
:100AC0007B347D347F347F34C43464340134013466
:100AD0001134003401341134003400340034003453
:100AE0000034003400340034003400340034003466
:100AF0000034003400340034003400340034003456
:100B00007F347E347C347B347A3479347734763471
:100B1000753474347234713470346E346D346C34B2
:100B20006B346934683467346634643463346234F3
:100B300061345F345E345D345B345A345934583434
:100B40005634553454345334513450344F344D3476
:100B50004C344B344A3448344734463445344334B7
:100B6000423441343F343E343D343C343A343934F9
:100B700038343734353434343334323430342F3439
:100B80002E342C342B342A3429342734263425347B
:100B900024342234213420341E341D341C341B34BC
:100BA00019341834173416341434133412341134FD
:100BB0000F340E340D340B340A3409340634053442
:100BC0000434033401340034C43464340134013453
:100BD0002234003401342234003400340034003430
:100BE0000034003400340034003400340034003465
:100BF0000034003400340034003400340034003455
:100C000080340034003401340234033404340634B4
:100C100008340A340C340E341134143417341A34B2
:100C20001D342134243428342C342F3433343734D5
:100C30003B343F34433447344B344F3452345634CE
:100C40005A345D346134643467346A346D347034DA
:100C500072347434763478347A347B347C347D3432
:100C60007E347E347E347E347E347D347C347B34FA
:100C70007A34783476347434723470346D346A343F
:100C80006734643461345D345A34563452344F34EA
:100C90004B34473443343F343B34373433342F34CC
:100CA0002C342834243421341D341A3417341434A9
:100CB00011340E340C340A3408340634043403344A
:100CC0000234013400340034C43464340134113447
:100CD00044340034013444340034003400340034EB
:100CE0000034003400340034003400340034003464
:100CF0000034003400340034003400340034003454
:100D000080340034003401340234033404340634B3
:100D100008340A340C340E341134143417341A34B1
:100D20001D342134243428342C342F3433343734D4
:100D30003B343F34433447344B344F3452345634CD
:100D40005A345D346134643467346A346D347034D9
:100D500072347434763478347A347B347C347D3431
:100D60007E347E347E347E347E347D347C347B34F9
:100D70007A34783476347434723470346D346A343E
:100D80006734643461345D345A34563452344F34E9
:100D90004B34473443343F343B34373433342F34CB
:100DA0002C342834243421341D341A3417341434A8
:100DB00011340E340C340A34083406340434033449
:100DC0000234013400340034C43464340134413416
:100DD0008834003401348834003400340034003462
:100DE0000034003400340034003400340034003463
:100DF0000034003400340034003400340034003453
:100E00003C1C08006C146D14EB011430B600071084
:100E10000130EB0507308A006B088207102F172F6F
:100E20006108F5006008F6000516D6011A2F7F301C
:100E3000D6001A2F701A432F6B18232F7019F60A39
:100E40007018F603272F7019F50A7018F503503043
:100E50007018EC007019ED00C8307602C830031825
:100E6000F600503076025030031CF600F51F3E2F7E
:100E7000A0307502A030031CF500432F64307502CA
:100E800064300318F5007F30D6006B1CD601B82201
:100E9000EA017927701C4E2F6D1B7016701D522FA2
:100EA0006C1B7016701E572FEB0A6B1C682F0710F7
:100EB000B60B5F2F07143C306B180A30B600640085
:100EC0000A300F02031C5F2F8F01701A082F1A2F90
:100ED0007508E1007608E000603084000408BB007B
:100EE0000008BA006221840A68300402031C6E2FD5
:100EF0000800F0010A30851DEC078519EC027830F6
:100F00006C020319701479300318EC0015306C0270
:100F10000319F0141430031CEC000A30051CED0713
:100F20000518ED0278306D02031970157930031839
:100F3000ED0015306D020319F0151430031CED009F
:100F40000800F1010A30871DEE0702308719EE0212
:100F500078306E020319711479300318EE001530E1
:100F60006E020319F1141430031CEE000A30071E40
:100F7000EF070230071AEF0278306F02031971157C
:100F800079300318EF0015306F020319F115143092
:060F9000031CEF00080045
:084000000A00030004000700A0
:02400E00CC33B1
:10420000010003000300030003000200020002009B
:1042100002000000000000000000FF00FF00FF009F
:10422000000000000000000000000000000000008E
:104230000000C000C000C000C000FF00FF00FF0081
:104240000100C300F300CF00FF00C300F300CF0064
:10425000FF00C300F300CF00FF00FF00FF00FF00DE
:10426000FF00FF00FF00FF00FF00FF00FF00FF0056
:10427000FF00FF00FF00FF00FF00FF00FF00FF0046
:10428000FF00FF00FF00FF00FF00FF00FF00FF0036
:10429000FF00FF00FF00FF00FF00FF00FF00FF0026
:1042A000FF00FF00FF00FF00FF00FF00FF00FF0016
:1042B000FF00FF00FF00FF00FF00FF00FF00FF0006
:1042C0007D00FC007D00FC007D00FC007D00FC000A
:1042D000FF00FF00FF00FF00FF00FF00FF00FF00E6
:1042E0000000000000000000FF00FF00FF00FF00D2
:1042F000FF00FF00FF00FF00FF00FF00FF00AA001B
:00000001FF
